:020000020000FC
:100000004DC0FFB6989B39C01123B1F4B29B29C0F3
:020010000AC024
:10001600FFB6112789B3807F8BBB882789BF37C07E
:10002600962CA72CB82C662477248824CC24DD248F
:10003600EE24B29B07C013959EEC92BF81E088BF69
:1000460081E089BF123060F069F0143020F031F49D
:100056009091690008C09B2D906205C0992703C046
:10006600992D01C09A2DB29992959F7089B3807F80
:10007600982B08C099B3907FB29B03C08FEF9F6007
:1000860002C09229812D9BBB88BB92E0B29B93E074
:1000960095BFFFBE189521E02EBF2FE52DBF2FEF90
:1000A6002ABB2BE027BB20E42BBF23E023BF0BD3C7
:1000B60060E0D7D1BFD1F8946FEFD3D12FEF28BB33
:1000C6002BBBB8D1222723BB2093680009D380F32A
:1000D60060E0C7D100FDD9D001FDE8D002FD30D1E6
:1000E60004FDD8D005FDF0D0202F2295022B6624E2
:1000F6007724882455243324442413D093E095BFD1
:1001060078949FD1889400FD36D040F001FD43D00D
:1001160028F002FD20D010F004D0F2CF2E3081F767
:10012600CACF98990BC0242D6FEF26272F70222E49
:1001360069B3607F262BB29B2BBB03C06C2C7D2C36
:100146008E2C232D25296FEFB29968BB2627B29BEB
:1001560028BB122E089520916E002A9519F020933F
:100166006E00089520917B0020936E00F4D1C8F3B1
:10017600C1F331D11FC020916E002A9519F020934A
:100186006E00089520916C0020936E00E4D1C8F3B0
:10019600C1F3EED00FC020916F002A9519F020937D
:1001A6006F00089520916D0020936F00CFD1C8F3A2
:1001B600C1F303D0989488940895989A2091680082
:1001C60021FD9898B0E0A7E822E099992D91223078
:1001D60009F008952D91662720FD626021FD61607A
:1001E600562E2695269536D0209369009B992D91FB
:1001F6009C9911C09A9918C0CD90DD902D912AD066
:100206002F70E22E2C2D219525D0C22E2D2D219535
:1002160021D0D22E08956D912D9129D0C62E6D91A3
:100226002D9125D0D62EEACF6D912C912F7023FDDE
:10023600206F1DD0C62E6D9162956F705C915295A0
:10024600507F652B2D9122952F7023FD206F0FD0A7
:10025600D62ED4CF222351F0622F2A7A60FD246055
:1002660062FD216064FD206466FD2061089527FD1E
:1002760006C0222311F467FF08956FE708952F3F04
:1002860011F467FD089560E8089520917900509172
:100296007B0004C020917A0050917C0020936A0074
:1002A60050936C0050936E0020E05DC02091790061
:1002B60020936B0020917B0020936D0020936F00AC
:1002C60060917D0068D10DC020917A0020936B006B
:1002D60020917C0020936D0020936F0060917E003A
:1002E60057D109F0089550917400EFE7F0E05523D7
:1002F60031F15A952191253811F4999A1AC0253968
:1003060031F45A952191203191F79B9AF0CF2537F8
:1003160039F45A952191203179F02C3079F0E7CFD4
:10032600237029F32A9529F02A9509F008C05A95D1
:1003360021915A952191DBCF9C9A08959A9A089516
:100346002091790020936A0020917B0020936C0015
:1003560020936E000895609181006933D9F762E0B9
:100366002091680026272093680021FD9898B0C048
:10037600F2DFB0E0AFE760E02C912F7009F061E0AA
:100386002D91207F09F062E0362E2D9133276627C6
:1003960008D0622BA738E0F3462E232D232B322ECE
:1003A60008955D912227583591F05A3291F05C32CA
:1003B60071F028E05F5451F021E05A9539F022E0BF
:1003C6005A9521F024E05A9509F0222708953260C3
:1003D600089531600895209180002F3739F02091DB
:1003E6008400259522956091850009C0209184009E
:1003F6002F702F30A1F320918400622F2295262B97
:100406002370662720FD626021FD6160362E60E064
:1004160020918300203009F464602F3F09F4626064
:1004260020918200203009F461602F3F09F4686052
:10043600462E089532E303D03A95E9F7089544E647
:1004460001C04AE003D04A95E9F7089524E6000082
:1004560000000000000000002A95C9F7089523E077
:10046600F6CF78EA7260DF987FB920D06FB91ED0D8
:10047600DF9A08957260DF987FB918D02D9115D054
:100486005A95E1F7DF9A0895DF987FB90FD02227B2
:1004960015D0DF9A0895DF987FB908D022270ED0AD
:1004A6002D935A95D9F7DF9A08952FB920E42EB9DE
:1004B6003BE13DB92EB126FFFCCF08952FB920E4CC
:1004C6002EB93BE13DB92EB126FFFCCF2FB10895E1
:1004D600F8E0EAE261E083D170E258E0CBDF60E465
:1004E60078EEC0DF20E120937000B4D009F00895C3
:1004F60060E878EEB7DF2227209371002093720020
:1005060003C060E078E3AEDF6091680070E1AADFC7
:1005160061E078E3A7DF20E220937000C6D009F4FB
:100526000895243041F420917100239520937100A1
:10053600283C39F709C02E3039F4209172002395F2
:10054600209372002530E9F622230895A7E8B0E04B
:1005560020916B0004C0AFE7B0E020916A002093C1
:100566007000A3D029F0243011F00894089508955E
:1005760070E38ADF522F2F9378E086DF2D935A950A
:10058600D9F778EC64E06EDF2F91222388940895E2
:10059600F8E0EAE409C0F8E0E2E406C0F8E0EAE3DD
:1005A60003C062E1F8E0E2E31AD170E258E062DFEC
:1005B60020E1209370004ED009F0089578EE60E2B5
:1005C600609377004FDF2E912E9106D021F420EA1A
:1005D600209370003FC00895AFE7B0E02093760007
:1005E60022272093740020E02093700033D009F076
:1005F600089570E349DF20937300522F78E044DFBB
:100606002D935A95D9F778EC64E02CDF209174008D
:1006160050917300250F2093740020917500521796
:1006260030F020917400509176002517E0F22227D1
:100636000895F8E0E2E2D2D0A0E6B0E070E258E039
:1006460019DF20E12093700005D009F0089520E815
:10065600209370002227209371002093720025D0EA
:1006660009F40895243041F42091710023952093D4
:100676007100283CA1F709C02E3039F42091720090
:10068600239520937200253051F7263061F460914E
:100696007700603111F060E101C060E2609377009D
:1006A60078EEE0DEE1F6222308956091700070EFA7
:1006B600D9DE78ECE9DE2078E1F360E8D3DE78EF86
:1006C600E3DE2F70089578E864E1CCDE78E760E237
:1006D600C9DE60E0C7DE78E6D7DE2170E9F308956B
:1006E60035D090F158EC86D04CD071F55ADF61F5D3
:1006F60068E054DF49F56091810050DF3091830056
:10070600E8E8F0E00781002309F404E0208920935B
:100716007D0024892F7020937900208D20937B0003
:10072600313079F0E1EAF0E027812295022B208929
:1007360020937E0024892F7020937A00208D2093A9
:100746007C0077DF889408950894089578ED61EC2D
:1007560089DE78EC60E286DE78EE64E083DE78EFB0
:1007660093DE207C61F078ED203821F06BEC7ADEA8
:10077600189403C069EC76DE9894889408950894DA
:10078600089528E02093750078EE61E06BDE78EE40
:100796007BDE2170E1F758EC2DD060E070EE62DE72
:1007A60068E000DF09F00895209186002093750027
:1007B60078EE61E057DE78EE67DE2170E1F758ECFF
:1007C60019D0F8E0E2E137DF09F008955EE112D0D2
:1007D60061E070EE47DEF8E0EAE12DCF662707D04C
:1007E60058E025912D935A95E1F75E936E93B0E00C
:1007F600A0E6089578EC60E435DE78EC45DE2074FA
:10080600E1F360E42FDE5A95C1F708950005010073
:10081600000000000009010000000000210A00009D
:10082600000000002109000200000100800600010E
:1008360000001200800600020000800081060022EF
:0C084600000080008106002201008000FC
:100FC0004D756C746948494431207665722E322E15
:100FD0003120202031302E30322E323032300D0A86
:100FE000415454696E7934342F3438202020202025
:100FF000202020202020286329206361726F0D0AA1
:00000001FF
